:100000000C948F000C94B7000C94B7000C94B700BC
:100010000C94B7000C94B7000C94B7000C94B70084
:100020000C94B7000C94B7000C94B7000C94B70074
:100030000C94B7000C94B7000C94B7000C94B70064
:100040000C9460030C94B7000C94FB040C944905C9
:100050000C94B7000C94B7000C94B7000C94B70044
:100060000C94B7000C94B70008000000BE9224491D
:10007000123EABAAAA2ABECDCCCC4C3E00000080DA
:10008000BEABAAAAAA3E00000000BF000000803F4D
:100090000000000000084178D3BB4387D1133D190D
:1000A0000E3CC3BD4282AD2B3E68EC8276BED98F3A
:1000B000E1A93E4C80EFFFBE01C4FF7F3F0000007E
:1000C000000000000000240027002A0000000000BB
:1000D000250028002B000000000023002600290036
:1000E00004040404040404040202020202020303DE
:1000F00003030303010204081020408001020408E6
:100100001020010204081020000000070002010076
:10011000000304060000000000000000AC061124EB
:100120001FBECFEFD8E0DEBFCDBF11E0A0E0B1E051
:10013000EEEFF8E102C005900D92A837B107D9F7AC
:1001400012E0A8E7B1E001C01D92AB32B107E1F7C0
:1001500011E0CEE1D1E004C02297FE010E94790CAB
:10016000CC31D107C9F70E9402070C947D0C0C9486
:100170000000AF92BF92CF92DF92EF92FF920F9367
:100180001F935A016B01AA2797FDA095BA2FBC01B6
:10019000CD010E947A0A7B018C0120E030E040E82A
:1001A00054E40E9476099B01AC01C601B5010E948E
:1001B000730BA80197010E94DF0990581F910F91BE
:1001C000FF90EF90DF90CF90BF90AF9008950F9386
:1001D0001F93CF93DF9300E010E0C0E0D0E080E019
:1001E0000E944504C80FD91F0F5F1F4F0031110532
:1001F000B1F7CE0160E170E00E942E0CCB01DF91DF
:10020000CF911F910F9108954F925F926F927F92BD
:100210008F929F92AF92BF92CF92DF92EF92FF9216
:100220000F931F93DF93CF9300D000D0CDB7DEB7ED
:100230002B013C0129833A834B835C8389E0882E20
:1002400082E0982EC40160E071E00E946309C4015D
:1002500064E171E00E946608C401B301A20122E0DA
:1002600030E00E945009C40161E271E00E9466081A
:10027000C40149815A816B817C8122E030E00E9477
:100280005009C40166E271E00E946608C401B80129
:10029000A70122E030E00E945009C4016BE271E046
:1002A0000E946608C401B601A50122E030E00E9468
:1002B0005009C301B20129813A814B815C810E94BE
:1002C000DF090E94330B3B014C0160E070E080E8E5
:1002D0009FE3A80197010E94DF097B018C0160E088
:1002E00070E080E89FE3A60195010E94DF09A40168
:1002F00093010E94730B9B01AC01C801B7010E94DE
:1003000077099B01AC0160E070E080E89FE30E9408
:10031000DF090F900F900F900F90CF91DF911F91F9
:100320000F91FF90EF90DF90CF90BF90AF909F9094
:100330008F907F906F905F904F900895AF92BF9293
:10034000CF92DF92EF92FF920F931F9320E030E560
:1003500043E457E40F2EF3E3EF2EF3E1FF2EF5E92C
:100360000F2FF3E41F2FF02D0F2EF0E0AF2EF0EE45
:10037000BF2EF6E7CF2EF5E4DF2EF02D0E9404010C
:100380001F910F91FF90EF90DF90CF90BF90AF90B3
:1003900008956F927F928F929F92AF92BF92CF9269
:1003A000DF92EF92FF920F931F935C0140E058E9B8
:1003B00067E377E40E94B9006B017C010E949E0113
:1003C000962E872E782E692E09E012E0C80164E18E
:1003D00071E00E946608C801B701A60122E030E082
:1003E0000E945009C8016FE271E00E946608C801CE
:1003F000B5014AE050E00E944708C80167E371E098
:100400000E946608C801292D382DE72DF62DA90177
:10041000BF0122E030E00E945009292D382D472DE0
:10042000562DB901CA011F910F91FF90EF90DF90F7
:10043000CF90BF90AF909F908F907F906F900895D6
:100440008E5F90E0611191E0692F0E94A6040895EB
:10045000CF93DF93C0E0D0E0CE0161E00E942002A4
:100460002196C930D105C1F7DF91CF910895EF9260
:10047000FF920F931F938C0189E092E060E471E09A
:100480000E946608B80180E090E00E94780A20E0AF
:1004900030E040E151E40E94730B20E030E040EA9C
:1004A00052E40E94760920E030E040EA51E40E94E4
:1004B000DF09AB01BC0189E092E022E030E00E945C
:1004C0004D0989E092E067E471E00E94630989E0E8
:1004D00092E069E471E00E94660889E092E0B80168
:1004E0004AE050E00E94EA0781E00031180718F066
:1004F0000E94280280C00F3F1105C1F1B8F1102FF2
:100500001F5FEE24E394E12280E090E06E2D0E94D4
:10051000200232E0F32EF12281E090E06F2D0E9464
:100520002002012F047082E090E0602F0E942002E0
:10053000187083E090E0612F0E94200284E090E038
:1005400061E00E94200285E090E06E2D0E94200272
:1005500086E090E06F2D0E94200287E090E0602FFF
:100560000E94200288E090E0612F43C0F02E602FAF
:10057000617080E090E00E942002602F627081E054
:1005800090E00E942002602F647082E090E00E9460
:100590002002602F687083E090E00E94200260E0FB
:1005A000C80124E0969587952A95E1F78F709070A1
:1005B0000F7010708017910708F461E084E090E0FC
:1005C0000E9420026F2D607885E090E00E9420025A
:1005D0006F2D607486E090E00E9420026F2D6072A3
:1005E00087E090E00E94200280E1F82288E090E01D
:1005F0006F2D0E9420021F910F91FF90EF900895A0
:100600000E94E7000E94C90123E333E948E853E46C
:100610000E94760920E030E040EA51E40E94770928
:1006200020E030E040E850E40E94730B0E944C0A46
:10063000DC01CB010E94370260E177E280E090E0CC
:100640000E94B403089589E092E040E05BE460E03A
:1006500070E00E94840582E061E00E94670483E00C
:1006600061E00E94670484E061E00E94670485E025
:1006700061E00E94670486E061E00E94670487E011
:1006800061E00E94670488E061E00E94670489E0FD
:1006900061E00E9467048AE061E00E9467048BE0E9
:1006A00060E00E9467048CE060E00E9467048BE0D9
:1006B00061E00E94A6048CE061E00E94A604089517
:1006C0001F920F920FB60F9211242F933F934F93C7
:1006D0005F936F937F938F939F93AF93BF9320917B
:1006E0007C0130917D0140917E0150917F0170919C
:1006F0008001DA01C9014096A11DB11D672F605D1F
:100700006D3730F06D57DA01C9014196A11DB11D59
:100710006093800180937C0190937D01A0937E0182
:10072000B0937F018091780190917901A0917A0135
:10073000B0917B010196A11DB11D8093780190932A
:100740007901A0937A01B0937B01BF91AF919F9102
:100750008F917F916F915F914F913F912F910F906A
:100760000FBE0F901F9018959B01AC017FB7F894B6
:100770008091780190917901A0917A01B0917B01EB
:1007800066B5A89B05C06F3F19F00196A11DB11D6C
:100790007FBFBA2FA92F982F8827860F911DA11DE3
:1007A000B11D66E0880F991FAA1FBB1F6A95D1F77C
:1007B000BC012DC0FFB7F894809178019091790128
:1007C000A0917A01B0917B01E6B5A89B05C0EF3FEF
:1007D00019F00196A11DB11DFFBFBA2FA92F982FA7
:1007E00088278E0F911DA11DB11DE6E0880F991F6E
:1007F000AA1FBB1FEA95D1F7861B970B885E934013
:10080000C8F2215030404040504068517C4F211583
:1008100031054105510571F60895789484B58260DB
:1008200084BD84B5816084BD85B5826085BD85B594
:10083000816085BDEEE6F0E0808181608083E1E843
:10084000F0E01082808182608083E0E8F0E08081C7
:1008500081608083E1EBF0E0808184608083E0EB65
:10086000F0E0808181608083EAE7F0E0808184604D
:1008700080838081826080838081816080838081A9
:10088000806880831092C1000895982F8E3008F000
:100890009E509770809167018295880F880F807CA9
:1008A000892B80937C0080917A00806480937A0009
:1008B00080917A0086FDFCCF2091780040917900EC
:1008C000942F80E030E0282B392BC9010895CF9375
:1008D000DF93482F50E0CA018C509F4FFC013491A8
:1008E00040525F4FFA018491882369F190E0880FAC
:1008F000991FFC01EE53FF4FA591B491FC01E45305
:10090000FF4FC591D491662351F42FB7F8948C9181
:10091000932F909589238C93888189230BC0623013
:1009200061F42FB7F8948C91932F909589238C9331
:100930008881832B88832FBF06C09FB7F8948C9142
:10094000832B8C939FBFDF91CF910895482F50E068
:10095000CA01885F9E4FFC012491CA018C509F4FB1
:10096000FC01949140525F4FFA013491332309F412
:1009700040C0222351F1233071F0243028F421307B
:10098000A1F0223011F514C02630B1F02730C1F0AB
:100990002430D9F404C0809180008F7703C0809107
:1009A00080008F7D8093800010C084B58F7702C057
:1009B00084B58F7D84BD09C08091B0008F7703C05E
:1009C0008091B0008F7D8093B000E32FF0E0EE0FB8
:1009D000FF1FE453FF4FA591B4912FB7F8946623FE
:1009E00021F48C919095892302C08C91892B8C9352
:1009F0002FBF089508951F920F920FB60F921124E2
:100A00002F933F934F938F939F93EF93FF938091F7
:100A1000C00082FD1DC04091C6002091C1013091EF
:100A2000C2012F5F3F4F2F7330708091C3019091AF
:100A3000C4012817390771F0E091C101F091C2019A
:100A4000EF57FE4F40833093C2012093C10102C093
:100A50008091C600FF91EF919F918F914F913F91AF
:100A60002F910F900FBE0F901F901895E0911502D7
:100A7000F0911602E05CFF4F8191919120813181CC
:100A8000821B930B8F739070892B11F00E94FA04D4
:100A900008951F920F920FB60F9211242F933F9338
:100AA0008F939F93EF93FF9320910502309106025D
:100AB00080910702909108022817390731F480913C
:100AC000C1008F7D8093C10014C0E0910702F091B6
:100AD0000802EB53FE4F208180910702909108029B
:100AE00001968F7390709093080280930702209371
:100AF000C600FF91EF919F918F913F912F910F90A1
:100B00000FBE0F901F901895AF92BF92DF92EF9299
:100B1000FF920F931F93CF93DF93EC017A018B0128
:100B2000DD24D39491E0A92EB12CEC89FD89DD2040
:100B300069F0C50108A002C0880F991F0A94E2F766
:100B4000808360E970ED83E090E005C0108268E486
:100B500078EE81E090E0A80197010E94410C2150BD
:100B6000304040405040569547953795279580E155
:100B70002030380720F0DD2011F0DD24D6CFE889C1
:100B8000F9893083EA89FB89208319A2EE89FF89DC
:100B9000408121E030E0C9010C8C02C0880F991F10
:100BA0000A94E2F7482B4083EE89FF894081C9010E
:100BB0000D8C02C0880F991F0A94E2F7482B4083DE
:100BC000EE89FF894081C9010E8C02C0880F991FF0
:100BD0000A94E2F7482B4083EE89FF8980810F8CCD
:100BE00002C0220F331F0A94E2F7209528232083A6
:100BF000DF91CF911F910F91FF90EF90DF90BF9009
:100C0000AF900895DC011C96ED91FC911D97E05C7E
:100C1000FF4F2191319180819181281B390B2F73D6
:100C20003070C9010895DC011C96ED91FC911D976F
:100C3000E05CFF4F20813181E054F040DF01AE5B8A
:100C4000BF4F8D919C9111972817390719F42FEFF9
:100C50003FEF07C08D919C91E80FF91F8081282FED
:100C600030E0C9010895DC011C96ED91FC911D97BF
:100C7000E05CFF4F20813181E054F040DF01AE5B4A
:100C8000BF4F8D919C9111972817390719F42FEFB9
:100C90003FEF10C08D919C911197E80FF91F2081B3
:100CA0008D919C91119701968F73907011969C93E2
:100CB0008E9330E0C9010895DC0191968C91919753
:100CC000882339F05496ED91FC915597808186FFE9
:100CD000F9CF91961C920895CF93DF93EC01EE85A6
:100CE000FF85E05CFF4F20813181E054F0402F5FB1
:100CF0003F4F2F733070DF01AE5BBF4F8D919C91E2
:100D0000119728173907D1F3E05CFF4F808191815B
:100D1000E054F040E80FF91F6083EE85FF85E05C4A
:100D2000FF4F31832083EE89FF89208181E090E0AD
:100D30000F8C02C0880F991F0A94E2F7282B20839A
:100D400081E089A3EC89FD8980818064808381E0D2
:100D500090E0DF91CF91089510920C0210920B0257
:100D600088EE93E0A0E0B0E080930D0290930E0235
:100D7000A0930F02B09310028CE691E090930A02C8
:100D80008093090281E891E0909316028093150206
:100D900085EC91E0909318028093170285EC90E027
:100DA00090931A028093190284EC90E090931C02B5
:100DB00080931B0280EC90E090931E0280931D02B2
:100DC00081EC90E09093200280931F0282EC90E0EF
:100DD000909322028093210286EC90E0909324026B
:100DE0008093230284E08093250283E0809326028F
:100DF00087E08093270285E08093280281E080933A
:100E000029020895CF93DF930E940D040E942303CB
:100E1000C6E3D5E00E9400032097E1F30E94360567
:100E2000F9CFCF92DF92EF92FF920F931F93CF9360
:100E3000DF937C016B018A01C0E0D0E00FC0D601D6
:100E40006D916D01D701ED91FC910190F081E02D44
:100E5000C7010995C80FD91F015010400115110590
:100E600071F7CE01DF91CF911F910F91FF90EF901D
:100E7000DF90CF900895EF92FF920F931F938C0114
:100E8000DC01ED91FC910190F081E02D6DE0099580
:100E90007C01D801ED91FC910190F081E02DC80119
:100EA0006AE009959C012E0D3F1DC9011F910F910C
:100EB000FF90EF900895CF93DF93EC0161157105DA
:100EC00019F420E030E00FC0DB010D900020E9F7BD
:100ED0001197A61BB70BE881F9810280F381E02D01
:100EE000AD0109959C01C901DF91CF9108954F9201
:100EF0005F927F928F929F92AF92BF92CF92DF923A
:100F0000EF92FF920F931F93DF93CF93CDB7DEB78E
:100F1000A1970FB6F894DEBF0FBECDBF2C01742E83
:100F2000CB01223008F42AE019A231E2C32ED12CE1
:100F3000CC0EDD1E822E9924AA24BB24672D752F8A
:100F4000A50194010E94410C79018A01C801B701F1
:100F5000A50194010E940F0C472D461B0894C1085F
:100F6000D1084A3014F4405D01C0495CF601408369
:100F7000E114F1040105110521F07E2C5F2DC8015B
:100F8000DDCFC201B6010E945B07A1960FB6F894AF
:100F9000DEBF0FBECDBFCF91DF911F910F91FF90AC
:100FA000EF90DF90CF90BF90AF909F908F907F9009
:100FB0005F904F900895DC012115310541F4ED91CA
:100FC000FC910190F081E02D642F099508950E9415
:100FD00077070895CF92DF92EF92FF920F931F93BE
:100FE0006C017B019A0100E010E0B801A7010E94AA
:100FF000DB078C01C6010E943B07080F191FC801BF
:101000001F910F91FF90EF90DF90CF900895CF92B6
:10101000DF92EF92FF920F931F93CF93DF93EC0138
:101020006A017B012115310541F4E881F9810190C4
:10103000F081E02D642F09951FC02A303105D1F4CD
:1010400077FF17C0E881F9810190F081E02D6DE212
:1010500009958C0144275527BA014C195D096E0981
:101060007F09CE012AE00E9477079801280F391FD7
:1010700004C02AE00E9477079C01C901DF91CF914B
:101080001F910F91FF90EF90DF90CF900895CF9236
:10109000DF92EF92FF920F931F936C017B019A01F5
:1010A0000027F7FC0095102FB801A7010E94070840
:1010B0008C01C6010E943B07080F191FC8011F9130
:1010C0000F91FF90EF90DF90CF9008950E945B0703
:1010D00008957F928F929F92AF92BF92CF92DF92AC
:1010E000EF92FF920F931F93CF93DF934C017A01FE
:1010F0008B01722ECB01BA01A80197010E94D60B79
:10110000882321F0C40169E571E021C0C0E0D0E08E
:1011100057016801E894D7F8C601B5012FEF3FEFFA
:101120004FE75FE70E94D60B882351F4C601B50153
:101130002FEF3FEF4FE75FE70E94DB09181614F02F
:10114000C1E0D0E0219739F0C4016DE571E00E9463
:101150005B07EC0193C0C801B7012FEF3FEF4FE7EA
:101160005FE40E942A0B181654F0C801B7012FEF54
:101170003FEF4FE75FEC0E94DB09882324F4C401B2
:1011800061E671E0E4CFC801B70120E030E040E063
:1011900050E00E94DB0987FD03C0C0E0D0E00EC034
:1011A000D401ED91FC910190F081E02DC4016DE23C
:1011B0000995EC0117FB109517F9109520E030E028
:1011C00040E05FE3DD240BC0CA01B90120E030E05C
:1011D00040E251E40E94DF099B01AC01D394D71493
:1011E00098F3C801B7010E9477095B016C010E9466
:1011F0004C0A7B018C01C401B801A7012AE030E050
:101200000E94DB07C80FD91F772039F0C40165E6BB
:1012100071E00E945B07C80FD91FC801B7010E9487
:10122000780A9B01AC01C601B5010E94760924C071
:1012300020E030E040E251E40E94730B7B018C011E
:101240000E94470A5B016C01CC24B7FCC094DC2CE3
:10125000C401B601A5012AE030E00E940708C80FCA
:10126000D91FC601B5010E947A0A9B01AC01C801D1
:10127000B7010E9476097A947720D1F6CE01DF91EA
:10128000CF911F910F91FF90EF90DF90CF90BF9083
:10129000AF909F908F907F9008950E946908089565
:1012A000EF92FF920F931F937C010E9469088C01BB
:1012B000C7010E943B07080F191FC8011F910F911A
:1012C000FF90EF900895EF92FF920F931F937C0190
:1012D0000E945B078C01C7010E943B07080F191F82
:1012E000C8011F910F91FF90EF9008955058BB27B0
:1012F000AA270ED075C166D130F06BD120F031F441
:101300009F3F11F41EF45BC10EF4E095E7FB51C161
:10131000E92F77D180F3BA1762077307840795071F
:1013200018F071F49EF58FC10EF4E0950B2EBA2FD4
:10133000A02D0B01B90190010C01CA01A0011124DB
:10134000FF27591B99F0593F50F4503E68F11A1687
:10135000F040A22F232F342F4427585FF3CF469518
:1013600037952795A795F0405395C9F77EF41F163A
:10137000BA0B620B730B840BBAF09150A1F0FF0F04
:10138000BB1F661F771F881FC2F70EC0BA0F621FF0
:10139000731F841F48F4879577956795B795F795E0
:1013A0009E3F08F0B3CF9395880F08F09927EE0F72
:1013B000979587950895D9D008F481E008950CD0C9
:1013C0000FC107D140F0FED030F021F45F3F19F09B
:1013D000F0C0511139C1F3C014D198F39923C9F366
:1013E0005523B1F3951B550BBB27AA27621773072B
:1013F000840738F09F5F5F4F220F331F441FAA1FDF
:10140000A9F333D00E2E3AF0E0E830D0915050409E
:10141000E695001CCAF729D0FE2F27D0660F771F4C
:10142000881FBB1F261737074807AB07B0E809F02E
:10143000BB0B802DBF01FF2793585F4F2AF09E3FC3
:10144000510568F0B6C000C15F3FECF3983EDCF395
:10145000869577956795B795F7959F5FC9F7880F3C
:10146000911D9695879597F90895E1E0660F771F8E
:10147000881FBB1F621773078407BA0720F0621B1F
:10148000730B840BBA0BEE1F88F7E095089504D018
:101490006894B111D9C00895BCD088F09F5790F0DE
:1014A000B92F9927B751A0F0D1F0660F771F881F89
:1014B000991F1AF0BA95C9F712C0B13081F0C3D0A4
:1014C000B1E00895C0C0672F782F8827B85F39F042
:1014D000B93FCCF3869577956795B395D9F73EF4E8
:1014E00090958095709561957F4F8F4F9F4F089590
:1014F000E89409C097FB3EF49095809570956195AE
:101500007F4F8F4F9F4F9923A9F0F92F96E9BB2763
:101510009395F695879577956795B795F111F8CFDF
:10152000FAF4BB0F11F460FF1BC06F5F7F4F8F4F4A
:101530009F4F16C0882311F096E911C0772321F040
:101540009EE8872F762F05C0662371F096E8862FD8
:1015500070E060E02AF09A95660F771F881FDAF72F
:10156000880F9695879597F90895990F0008550F5C
:10157000AA0BE0E8FEEF16161706E807F907C0F019
:1015800012161306E407F50798F0621B730B840B21
:10159000950B39F40A2661F0232B242B252B21F4FB
:1015A00008950A2609F4A140A6958FEF811D811D9B
:1015B000089597F99F6780E870E060E008959FEFD5
:1015C00080EC089500240A941616170618060906DA
:1015D000089500240A9412161306140605060895A9
:1015E000092E0394000C11F4882352F0BB0F40F431
:1015F000BF2B11F460FF04C06F5F7F4F8F4F9F4F71
:10160000089557FD9058440F551F59F05F3F71F0F2
:101610004795880F97FB991F61F09F3F79F0879559
:101620000895121613061406551FF2CF4695F1DFE2
:1016300008C0161617061806991FF1CF8695710572
:10164000610508940895E894BB2766277727CB01A6
:1016500097F908958ADF08F48FEF08950EF0AAC075
:10166000AECF6894A6CFD5DFC8F39923D1F3C6F3E4
:10167000DF93CF931F930F93FF92C92FDD2788230A
:101680002AF02197660F771F881FDAF720E030E0F5
:1016900040E85FEB9FE3883920F0803E30F02196F0
:1016A0008F7725DEE8E6F0E003C021DEE5E9F0E033
:1016B00091D08B01BE01EC01FB2E6F57710975951E
:1016C000771F880B990B16DF28E132E741E35FE3D0
:1016D00016D0AF2D9801AE01FF900F911F91CF91C1
:1016E000DF9116DE7DCF0BD07BCF6CDF28F071DF72
:1016F00018F0952309F05DCF62CF1124A5CF81DFCB
:10170000A0F3959FD1F3950F50E0551F629FF00114
:10171000729FBB27F00DB11D639FAA27F00DB11D6D
:10172000AA1F649F6627B00DA11D661F829F2227F6
:10173000B00DA11D621F739FB00DA11D621F839F7D
:10174000A00D611D221F749F3327A00D611D231F53
:10175000849F600D211D822F762F6A2F11249F57A1
:1017600050408AF0E1F088234AF0EE0FFF1FBB1FC4
:10177000661F771F881F91505040A9F79E3F510563
:1017800070F017CF61CF5F3FECF3983EDCF38695A6
:1017900077956795B795F795E7959F5FC1F7FE2B0E
:1017A000880F911D9695879597F90895DEDE880B31
:1017B000990B08959F3F49F0915028F486957795AD
:1017C0006795B7959F5F80389F4F880F969587954F
:1017D00097F90895DF93CF931F930F93FF92EF92A2
:1017E000DF927B018C01689405C0DA2EEF0187DF60
:1017F000FE01E894A5912591359145915591AEF35F
:10180000EF0186DDFE019701A801DA9479F7DF90F8
:10181000EF90FF900F911F91CF91DF910895629FFC
:10182000D001739FF001829FE00DF11D649FE00DD8
:10183000F11D929FF00D839FF00D749FF00D659F39
:10184000F00D9927729FB00DE11DF91F639FB00D38
:10185000E11DF91FBD01CF011124089597FB092E49
:1018600007260AD077FD04D02ED006D000201AF427
:10187000709561957F4F0895F6F7909581959F4FEC
:101880000895A1E21A2EAA1BBB1BFD010DC0AA1FC1
:10189000BB1FEE1FFF1FA217B307E407F50720F0D9
:1018A000A21BB30BE40BF50B661F771F881F991F54
:1018B0001A9469F760957095809590959B01AC019D
:1018C000BD01CF010895AA1BBB1B51E107C0AA1F90
:1018D000BB1FA617B70710F0A61BB70B881F991FD1
:1018E0005A95A9F780959095BC01CD010895EE0F0A
:0E18F000FF1F0590F491E02D0994F894FFCFAE
:1018FE00436F6D707574652074656D70657261747B
:10190E0075726500526573697374616E63653A2012
:10191E000052303A200054303A2000423A2000560D
:10192E00616C75653A20004B656C76696E3A2000E5
:10193E0054656D703A20004600456E636F646564B1
:10194E002076616C75653A20006E616E00696E6678
:10195E00006F7666002E0001000000006C06110775
:08196E000206330613065C06B5
:00000001FF
